:100000000AC023C022C021C020C01FC01EC01DC006
:100010001CC01BC01AC011241FBECFEDCDBF10E005
:10002000A0E6B0E0E2E1F2E003C0C89531960D929F
:10003000A036B107D1F710E0A0E6B0E001C01D92F4
:10004000A036B107E1F7A4D0E3C0DACFCF93DF93B6
:10005000CDB7DEB7E8E3F0E01082E7E3F0E080E15F
:100060008083E2E3F0E01082E1E3F0E08AE0808365
:10007000DF91CF910895CF93DF93CDB7DEB725976A
:100080000FB6F894DEBF0FBECDBF6A837B838C832F
:100090009D838A819B81AC81BD81880F991FAA1F96
:1000A000BB1F880F991FAA1FBB1F880F991FAA1F6C
:1000B000BB1F880F991FAA1FBB1F282F392F4A2F3C
:1000C0005B2F80E896E9A8E9B0E0682F792F8A2FA6
:1000D0009B2F77D0B52FA42F932F822F8150898308
:1000E000E9E2F0E089818083AAE2B0E0EAE2F0E0B0
:1000F000808188618C9325960FB6F894DEBF0FBE81
:10010000CDBFDF91CF910895CF93DF93CDB7DEB709
:1001100022970FB6F894DEBF0FBECDBFEBE2F0E042
:100120008081882344F4ECE2F0E08081282F33279B
:100130003A83298302C01A82198289819A81229680
:100140000FB6F894DEBF0FBECDBFDF91CF910895FB
:10015000CF93DF93CDB7DEB721970FB6F894DEBF0C
:100160000FBECDBF8983EBE2F0E0808199278072DA
:1001700090700097C1F3ECE2F0E0898180832196D2
:100180000FB6F894DEBF0FBECDBFDF91CF910895BB
:10019000CF93DF93CDB7DEB721970FB6F894DEBFCC
:1001A0000FBECDBF53DF60E875E280E090E063DF13
:1001B00000C0AADF898389818823D9F38981C8DFB8
:1001C000F8CFA1E21A2EAA1BBB1BEA2FFB2F0DC0F2
:1001D000AA1FBB1FEE1FFF1FA217B307E407F507F7
:1001E00020F0A21BB30BE40BF50B661F771F881FD3
:1001F000991F1A9469F76095709580959095262FB0
:10020000372F482F592F6A2F7B2F8E2F9F2F08951E
:02021000FFCF1E
:00000001FF
